:100000008A010F2801290F29212934293F29512943
:1000100088299829F229FB29042A142A272A022050
:100020008A110A1207208A110A123C308312AC008E
:1000300006208A110A120F308312AC0006208A11A2
:100040000A12831287011B308316870080309400C8
:1000500009309300283083129400A9018312AA0169
:10006000A501831225080F3C013003190301003C50
:100070000319932809208A110A12103083122502CD
:10008000013003180301003C03198728A908013037
:10009000031D0301003C0319862801308312A900C7
:1000A0000A302502013003180301003C03196228BD
:1000B000A0012508303E0318A00AAB0004208A11D5
:1000C0000A126C288312A0012508373E0318A00AE3
:1000D000AB0004208A110A120A208A110A12A030E9
:1000E0008312AD000C208A110A1283122A08AD0077
:1000F0000C208A110A1283122508AD000C208A11E7
:100100000A120B208A110A128312AA0A8C2883125F
:10011000290803198C28A9010A308312A20008209B
:100120008A110A123128C0308312AC0006208A11CD
:100130000A128312AA010A208A110A12A03083121D
:10014000AD000C208A110A1283122A08AD000C207F
:100150008A110A120B208A110A120A208A110A1225
:10016000A1308312AD000C208A110A128312A5015E
:10017000831225080F3C013003190301003C0319C9
:10018000F7280D208A110A128312A5000A302502D1
:10019000013003180301003C0319D828A0012508E9
:1001A000303E0318A00AAB0004208A110A12E2288C
:1001B0008312A0012508373E0318A00AAB000420D3
:1001C0008A110A12831225080F3C0130031D030116
:1001D000003C0319F1280130AE000E208A110A12EA
:1001E000F6288312AE010E208A110A12B8280B20BD
:1001F0008A110A1202308312AC0006208A110A12F8
:100200002E2883128501F8308316850006309F0062
:100210008312051005118510831686010800FF3032
:1002200083168600831285148312051100000515BC
:100230000000861B14290511000085108316860115
:1002400008008312851005102B08860003208A11F0
:100250000A12831205140515000005112D30A400A3
:1002600005208A110A120800A40CA40C3F30A40532
:100270000330A4020000A40B3A29000008008312F6
:10028000851005102C08860003208A110A1283129B
:100290000515000005112D30A40005208A110A1251
:1002A00008003C308312AC0006208A110A12053087
:1002B0008312A20008208A110A123C308312AC007B
:1002C00006208A110A1205308312A20008208A1122
:1002D0000A123C308312AC0006208A110A12053043
:1002E0008312A20008208A110A1208308312AC007F
:1002F00006208A110A1201308312AC0006208A11EE
:100300000A1206308312AC0006208A110A12080075
:100310008E308312A30000000000000000000000E7
:100320000000A30B8D290000A20B88290000080003
:10033000F030831686008113831286010609A70018
:10034000A70EA601831227080139FF390130031DCA
:100350000030003C0319B129270C7F39A700A60AF9
:10036000A229043083122602013003180301003C45
:100370000319EE292608A8000F3083168600811382
:10038000831286010609A700A601831227080139F6
:10039000FF390130031D0030003C0319D429270C1C
:1003A0007F39A700A60AC52904308312260201302E
:1003B00003180301003C0319EA292608A700A0013D
:1003C0002808A100A10D210DFC3927070318A00A58
:1003D000A500ED29FF308312A500F129FF3083121B
:1003E000A500080083128C11831611148316111CAA
:1003F000FA29F629080083128C1183161115831629
:10040000111D032AFF29080083128C112D08930067
:1004100083120C080839003C0130031D0301003C25
:100420000319132A082A080083128C1183169115C8
:1004300083120C080839003C0130031D0301003C05
:100440000319232A182A83128C1113080800831217
:100450008C112E08003C0319302A83169116322A7B
:10046000831691128316111683120C080839003C6A
:100470000130031D0301003C03193F2A342A080000
:00000001FF
